:020000040001F9
:10B00000A8220020D5B00100EFB00100F1B001008E
:10B010000000000000000000000000000000000030
:10B02000000000000000000000000000F3B001007C
:10B030000000000000000000F5B00100F7B00100C2
:10B040009DB30100F9B00100F9B00100B9B40100ED
:10B05000F9B001000000000019B20100F9B00100D0
:10B06000F9B00100F9B00100F9B00100F9B0010038
:10B07000F9B00100F9B00100F9B00100F9B0010028
:10B08000F9B00100F1B30100F9B00100F9B001001D
:10B09000CDB40100F9B00100F9B00100F9B0010030
:10B0A000F9B00100F9B0010000000000000000004C
:10B0B0000000000000000000000000000000000090
:10B0C0000348854600F096F80048004709C1010092
:10B0D000A82200200321094802680A4302600848A8
:10B0E00002680A4302600748804707480047FEE7B6
:10B0F000FEE7FEE7FEE7FEE7FEE70000240500406E
:10B1000054050040D5B40100C1B0010003460B4313
:10B110009B0703D009E008C9121F08C0042AFAD20D
:10B1200003E00B780370401C491C521EF9D2704793
:10B13000421C0178401C0029FBD1801A704703464D
:10B140000A780270401C491C002AF9D11846704741
:10B15000F0B51FB40646002082B005464024019198
:10B1600000901BE0019922460F46304600F030F86F
:10B17000049A059B801A994110D31046194622461D
:10B1800000F016F8361A8F4101972246012000215F
:10B19000009F00F00DF838184D4100902046641EC5
:10B1A0000028DFDC019B00982946324607B0F0BD3D
:10B1B00010B5202A04DB0146203A9140002010BD42
:10B1C000914020239C1A0346E3401943904010BD50
:10B1D00010B5202A04DB0846203AD040002110BDDB
:10B1E0000B46D340D0402024A21A91400843194670
:10B1F00010BD0000064C0125064E05E0E36807CCB3
:10B200002B430C3C98471034B442F7D3FFF75CFF54
:10B21000B4CA0100D4CA0100F0B50025FF2689B0E8
:10B22000013601242F460195304601F06BF80028C5
:10B2300007D044484068204203D0304601F05AF815
:10B240002543361D64007F1CB6B2042FECD3FF24C7
:10B250007D34204601F056F8002807D0204601F042
:10B2600049F860070543384800690190374C2807C2
:10B2700014D0012700262F420CD03548B2001118F7
:10B2800008690969C004C00E8903A258890F002A01
:10B2900000D090477F00761C042EECD3002D2FDACF
:10B2A0000020421E264620360590307D0027850668
:10B2B000AD0E41B2491C23D00121A9401142009199
:10B2C0001ED080090390284600F032FD80002058EF
:10B2D0000490002802D10398032811D10398009903
:10B2E000032802D10598084305901A4AA80080183F
:10B2F0000068019A8003800F114203D0022803D016
:10B3000009B0F0BD0328FBD10399032906D1022817
:10B3100015D00221284600F0DDFF012704980028FF
:10B3200003D0049A284603999047002FE8D0064896
:10B33000006901998842E3D00190059AB5E703219D
:10B34000E8E700000063004000050050701A00208C
:10B3500000650040000700508307FF22DB0E9A4083
:10B360008907090E994000280BDA0007000F0838FA
:10B37000830808489B001818C36993430B43C361B3
:10B380007047830804489B001B18186890430843C3
:10B390001860704700ED00E000E400E0F8B5FF2021
:10B3A000013000F0FBFE002401250E4E0E4F002858
:10B3B00007D00E4804600120B0607D70002000F0CE
:10B3C000BFFCFF20053000F0E9FE002808D0074848
:10B3D000001D04600220B060BD70012000F0B0FCD0
:10B3E000F8BD000000030040341A002000010040B6
:10B3F00010B506490020086048608860C8600349AD
:10B4000040390860486001F099F910BD40110140D1
:10B41000FFB5114F0446387881B01D461646002806
:10B4200001D100F0A7F83869A04211D918200A49C3
:10B4300060434118002C06D00298CE610D628861ED
:10B440000020886248620A98C862002005B0F0BDFA
:10B450000020C043FAE70000BC19002070B50E467A
:10B4600018214843134914464518E86A183500283E
:10B4700004D001280FD0022805D113E0284600F09F
:10B48000AFF8A04201D2002411E0224631462846FE
:10B4900000F0E1F80BE0284600F0A2F8A042F4D258
:10B4A0000446F2E73146284600F0A5F80446204657
:10B4B00070BD0000BC19002010B50249024800F020
:10B4C000C7FC10BD481A00200030004010B501F044
:10B4D000CBF810BD10B500F011FD002805D01F49B4
:10B4E0001D484860C8131E4988611E48018CC9B2B6
:10B4F00001290BD1828C120708D1028D1206120F7E
:10B50000042A03D1828D1206120F0AD0012921D1FB
:10B51000818C09071ED1018D0906090F0A2904D063
:10B5200007E0114A01219160F5E7828D1206120FA2
:10B5300005D00D290ED1808D0006000F0AD10B48D1
:10B540000168012904D00A49016001680129FCD180
:10B55000C021416110BD0000DFFF07C000050040B1
:10B56000006C0040C00F00F00006004000EC0640F8
:10B570007593000010B5124C02202061606111A08B
:10B58000A0611348E0610120800220620020A062D7
:10B5900060620CA1A1642146E0621039E1641021CF
:10B5A0002165A0656065E0650AA1E01DFFF7C7FDA4
:10B5B00009A12046FFF7C3FD2020A07110BD0000A7
:10B5C000BC1900205465726D696E616C000000004A
:10B5D000AC150020525454005345474745520000D3
:10B5E0000269C1688A4203D88068401A801800E066
:10B5F000501A401E7047F7B5064682B000200090F2
:10B60000F46817463069A04201D9051B02E0B16811
:10B61000201A0D1AB0686D1E001BA84200D80546FE
:10B62000BD4200D33D4670682A4600190399FFF7D2
:10B630006DFD00987F1B4019009003986419401914
:10B640000390B068A04200D10024F460002FD9D14B
:10B65000009805B0F0BDF7B5C66817460446806887
:10B66000851B6068BD4206D980190199FFF74EFD20
:10B67000F019E060FEBD2A4680190199FFF746FDEA
:10B6800001987E1B411932466068FFF73FFDE66076
:10B69000FEBD00000FB410B504A9074B02AA039821
:10B6A00000F028F8044602A9002000F05DFA2046C8
:10B6B00010BC08BC04B0184769BB010030B4744624
:10B6C000641E2578641CAB4200D21D46635D5B009E
:10B6D000E31830BC184702E008C8121F08C1002A4E
:10B6E000FAD170477047002001E001C1121F002A03
:10B6F000FBD17047FFB591B00F460546002606E026
:10B7000025280AD0149A139990476D1C761C287826
:10B710000028F5D1304615B0F0BD00240094012179
:10B72000F34A029400E004436D1C2B780846203B4A
:10B7300098401042F7D128782A280ED00221287884
:10B740000246303A092A15D8009A0A235A43303A59
:10B7500080180C436D1C0090F1E701CF0090002889
:10B7600005DA012040030443009840420090022083
:10B7700004436D1C28782E2815D1042004436878D2
:10B780006D1C2A280AD101CF6D1C02900BE0029992
:10B790000A225143303940186D1C02902878014626
:10B7A00030390929F3D928786C2810D006DC4C28C8
:10B7B0001AD068280ED06A2817D104E0742813D054
:10B7C0007A2812D110E00120400504430CE0012149
:10B7D000090501E0032109050C436978814203D181
:10B7E0000120000524186D1C6D1C287803906E281C
:10B7F0001ED00CDC632831D004DC00288AD0582805
:10B8000011D1B2E064287BD069280CD178E073288C
:10B810002DD004DC6F2870D0702804D1A7E07528E3
:10B820006CD078286BD0149A13999047761C62E0FC
:10B830006002400F022807D003280AD00428386885
:10B840000AD006603F1D56E03868F1170660416077
:10B85000F8E738680680F5E70670F3E73878694658
:10B8600008740020487404A80390012003E038689D
:10B8700003900020C0433F1D61070FD5002101E068
:10B880000199491C029A0191914213DA8142F7DB36
:10B89000019A0399895C0029F2D10BE0002101E0B3
:10B8A0000199491C01918142FADB019A0399895C53
:10B8B0000029F5D101990098139A401A0090214669
:10B8C000149B00F03BF901998019461807E0039892
:10B8D00003990078491C0391149A13999047019891
:10B8E000401E0190401CF2D12146149B139A0098EF
:10B8F00000F014F986196D1C09E741E033E034E0EB
:10B900000A200021049005916002410F022905D010
:10B9100001CFC2179446032905D007E0FF1DFF0899
:10B92000FF0003CF06E000B2C2179446042902D1FB
:10B9300040B2C1178C4600226146944506DA0A4699
:10B940000021404291418C462D2102E0210504D581
:10B950002B216A461176012103E0E10701D0202165
:10B96000F7E7019154E00A200BE0102009E01020D5
:10B97000049000210420044308200591029003E074
:10B9800008200021059104906002410F022905D092
:10B9900001CF00229446032906D006E0FF1DFF08D0
:10B9A000FF0003CF8C4603E080B2042900D1C0B26F
:10B9B0000021019121072BD50399702906D0049A03
:10B9C0001021059B4A401A4305D00EE040216A46EB
:10B9D0001176012108E06146014306D030216A4614
:10B9E00011760399517602210191049A0821059B51
:10B9F0004A401A430CD16146014301D1610707D582
:10BA000030216A461176012101910299491E029165
:10BA10000399582904D037A103910FA90F910DE084
:10BA200039A1F9E76146059B049AFFF791FB039B57
:10BA30008C469B5C0F9A521E0F9213706146014315
:10BA4000F0D10F9807A9081A20300390600704D599
:10BA5000012000048443029801E001200290039930
:10BA6000884201DD401A00E0002041180290019850
:10BA700009180098401A0090E00306D42146149B50
:10BA8000139A009800F05AF886190020049008E0F4
:10BA900006A9085C149A139990470498401C761CD8
:10BAA000049001998842F3DBE0030CD52146149BF6
:10BAB000139A009800F042F8861904E0149A302096
:10BAC00013999047761C0299481E02900029F5DCD4
:10BAD00008E00F980F990078491C0F91149A139958
:10BAE0009047761C0399481E03900029F1DCFBE681
:10BAF0000928010030313233343536373839616244
:10BB00006364656600000000303132333435363707
:10BB1000383941424344454600000000F8B5044628
:10BB200000251E461746880404D405E03946202027
:10BB3000B0476D1C641EF9D52846F8BDFFB5044614
:10BB4000002581B01E46C80301D5302700E020271C
:10BB5000880404D505E038460399B0476D1C641E7F
:10BB6000F9D5284605B0F0BD0A68531C0B6010706B
:10BB70007047000006A1012000F00EFDBFF34F8FBB
:10BB80000A490948C860BFF34F8F00BFFDE70000B6
:10BB90004150505F4552524F523A4552524F523ADD
:10BBA000466174616C0D0A000400FA0500ED00E0C6
:10BBB0000EB50021029000916A4601910148FFF7FD
:10BBC000D9FF0EBD01400000094B5B68002B07D078
:10BBD000002A07D0002805D00068037C002B03D082
:10BBE0000820704707207047417442610020704769
:10BBF000E4130020FFB507469007002581B01E46DC
:10BC00001446002825D1002C23D000F0F5FC304646
:10BC1000114EF06030461030057045700299817009
:10BC200044607560357001240C487570240504600B
:10BC300003211420FFF790FB09480460094CA7601A
:10BC400003211120FFF788FB6068B060002005B079
:10BC5000F0BD0720FBE70000D413002080E200E0E5
:10BC600000E100E000150140FEB51D4B5B68002BB4
:10BC70002DD000282BD0052901D20720FEBD436915
:10BC8000002B24D0437C012B23D000270446002521
:10BC900016462846019100F027F8684600F0F0FEAD
:10BCA000002818D0012101700E4944604968816064
:10BCB000019907614661C16068460949007848708A
:10BCC000002000F015F800F011FD2846FEBD082008
:10BCD000FEBD0F46DAE70425002000F009F8F4E77E
:10BCE000E41300200015014000B500F005F800BD88
:10BCF00000B500F009F800BD72B602480168491CA1
:10BD000001607047CC13002003490868401E08609A
:10BD100000D162B670470000CC130020002901DA80
:10BD20000020704702685118016001207047000030
:10BD3000024909181420085670470000701A0020A4
:10BD400070B5084C050009D010342168002907D0CF
:10BD500008682060496828468847F6E70834F4E711
:10BD600070BD0000341A0020F8B52348416800294E
:10BD70003ED00E6821494C6887688078E11B0D022F
:10BD80002D0AED1C002814D101201D4A000450602A
:10BD90001B4A403A50601B49400008601A4908603D
:10BDA0001A49012008602F2000F000FA12490120F2
:10BDB0008870B54200D23546E81900020F4B000AE0
:10BDC000403318600D4A5168001B091B0902090A1B
:10BDD0000002000AC91C814209D9506818602F204E
:10BDE00000F0E4F901200749400480390860F8BDFB
:10BDF00000F002FCF8BD0000D41300200015014043
:10BE00004013014080E200E000E100E0001001404A
:10BE100010B50E4900230A784C78A24212D0521C69
:10BE2000D2B20A70022A00D10B700A78074B920036
:10BE300018339A580260886810180002000A886057
:10BE4000012010BD0360002010BD0000D4130020AD
:10BE50007FB50C460D462035064669782878019155
:10BE6000009022462632D11E3046E36900F035FDAF
:10BE7000002819D1E87800281DD1207B022801D0A4
:10BE8000032818D12269E169914214D16269E26103
:10BE9000E37B2B70217E8906C90F6970032804D0CB
:10BEA0003146204600F0B2FC7FBD0091314620466D
:10BEB00000F098FD7FBD20460C3007C801AB07C3DA
:10BEC000E878002100280ED00920C0013218506CFB
:10BED0005064820701D5012002E0400705D5022009
:10BEE0006A46107001E0684601702971207E4007A3
:10BEF000E0D422686846616890477FBD1048018C95
:10BF0000C9B2012917D1818C090714D1018D090605
:10BF10000A0F03D1828D1206120F0ED0090F0129CC
:10BF200003D1828D1206120F07D0032903D1808D11
:10BF30000006000F01D0002070470120704700006C
:10BF4000C00F00F002680A600160704770B50B49CD
:10BF50004B680C4C0A482268855C0120A8400546C5
:10BF60009D438D601840C860521C9207920F06A135
:10BF70000320226000F016FB70BD00000005005099
:10BF8000B0CA0100C81300203A494E464F3A496EE4
:10BF900076657274696E67206C65642025640A009A
:10BFA000F0B5284C2146103948688B6822788646BF
:10BFB0009C46CF78667836E0182353436168521C5C
:10BFC000C918A378D2B2934200D100220B78022B79
:10BFD00002D0032B27D123E003464D68194603E026
:10BFE000A94204D00B46C96900291CD0F8E70029F2
:10BFF00019D08B4208D1C069002805D1124F012504
:10C00000BD600025AC4601270D68C969D9610029CA
:10C0100009D00B685B190B6005E00174C06900E092
:10C0200000210028F9D19642C6D10649624610394E
:10C030008A604860CF70704501D00120F0BD0020BB
:10C04000F0BD0000E413002000100140F8B52C4EB4
:10C05000044670680025009041E0002C02D0204684
:10C06000E46920E0264818231030017842684B43E9
:10C07000491CC9B2D21801708378994200D1057069
:10C080001178506801292CD1017C002929D19168AF
:10C090004160D16881601169C16051698161F17845
:10C0A000002900D045604368B268164F991A09020A
:10C0B000090AB94202D28268891806E0D11A090237
:10C0C0008268090A8A4202D9511A016000E00560BB
:10C0D0004560012185600174C56100F00FFB002CF3
:10C0E000BBD107481030017840788142BAD17168DD
:10C0F0000098814201D00120F8BD0020F8BD000069
:10C10000D4130020FFFF7F0000F068F8002801D062
:10C11000FFF74EFD002000F07BF8002000F050FA01
:10C12000002801D0FFF744FD0023184A05211846D6
:10C13000FFF760FD002801D0FFF73AFD144A012106
:10C140001448FFF741FD002801D0FFF731FD1148E9
:10C1500001210022C9030068FFF786FD002801D0F5
:10C16000FFF726FD002001210B4B03220C468440E3
:10C17000E401240F02D08400E4182260401C20282F
:10C18000F4D320BF40BF20BFFBE7000018140020FD
:10C190004DBF0100ACCA0100000700500121890712
:10C1A00040180068002800D00120704700280FD0F8
:10C1B0000849094A096800BF00BF00BF00BF00BFAF
:10C1C00000BF00BF00BF914200D000BF401EF2D1AF
:10C1D00070470000F41300200024F40010B50A4C4E
:10C1E0002078002801D0852010BD0020A06060606C
:10C1F0002061E060032100F03DF8044901208861DE
:10C200002070002010BD0000341A002000050040FE
:10C2100070B5154C0546A078002808D0002D02D036
:10C220006968012088470020FFF75EFD15E00020C7
:10C23000FFF75AFD002D04D00B4829461030FFF7B8
:10C2400081FEE068002808D10849086008490220FA
:10C25000486006490120FC390860E068401CE06045
:10C260000020FFF745FD70BD341A00200401004096
:10C27000000300408207D30EFF229A408907090E6F
:10C2800010B5994000280BDA03071B0F083B9C08E8
:10C290000C4BA400E318DC6994430C43DC6107E019
:10C2A0008408094BA400E418236893430B432360DC
:10C2B000C106C90E0120884004490860044908608D
:10C2C00010BD000000ED00E000E400E080E200E0CE
:10C2D00000E100E0820006481018026803231B04F6
:10C2E0009A430260026809040A4302607047000032
:10C2F000000700500249401800210160704700000B
:10C3000000600040034940180068012800D0002068
:10C3100070470000006000400048704765C301009E
:10C32000F8B50C4C05462078002804D0607885428A
:10C3300001D10020F8BD01263302074A07A10020E1
:10C340000096FFF765F8002801D00820F8BD267098
:10C350006570EEE7D0130020AC1400204E6F726DB4
:10C36000616C0000F0B5C3B01746084600224B9937
:10C370000092499A1C4651180291002801D00A21C6
:10C3800000E0002103AE0191002C15D131466A4630
:10C3900000F014FA00286AD03846FEF7C9FEC22819
:10C3A00000D9C220054600982A4630183946FEF7C3
:10C3B000ADFE0098401900900199009803AA411819
:10C3C000101831315118002203E020230370401C63
:10C3D000521C019B9A42F8D30026029A944207D33A
:10C3E00020220270427082700A70C01C491C26E034
:10C3F000499A944202D2489A125D02E0A31A4A9ADC
:10C40000D25C01259446AB006246DA4013071B0F4D
:10C41000092B01D9373300E0303301277F1B6D1E14
:10C42000C3556A1CEFD12022827062461346203B1E
:10C43000C01C5E2B00D92E220A70491C641C761C7D
:10C44000102ECAD30D220A700A224A7020210170D0
:10C45000009901980918433103A8009100F0EEF803
:10C46000002804D00020009002988442A4D32046E3
:10C4700043B0F0BDFFB5C5B00846002505AE1C466B
:10C480004E9F314604AA049500F098F900282FD059
:10C490003B00FFF713F90705131A2F38434F21000C
:10C4A0004798FEF745FE049905464018FF2813D823
:10C4B00070182A464799FEF729FE0DE00498226875
:10C4C00030184799FFF7E6F805E004980CCC3018CF
:10C4D0004799FFF7DFF80546294604A8FFF71EFC39
:10C4E000002804D0FF200499013081422ED9002079
:10C4F00049B0F0BDA068009004980CCC3018479962
:10C50000FFF7C8F8E7E7E168A06800900191049898
:10C510000CCC30184799FFF7BDF8DCE7204608300F
:10C5200007C86B4607C304980CCC30184799FFF72F
:10C53000B1F8D0E7204608300FC86D460FC5049803
:10C540000CCC30184799FFF7A5F8C4E705A800F010
:10C5500075F8CDE70048704775C40100FFB583B09A
:10C560000020084D019028691E46174601AC8047FF
:10C57000009601906D693B462146049A0398A847AE
:10C5800007B0F0BD9014002000B5024B1A6100F016
:10C5900011F800BD9014002010B500231A46FFF7D3
:10C5A000DDFF10BD08B5009201236A46FFF7D6FFF4
:10C5B00008BD0000014A916150617047901400204D
:10C5C00070B5050005D00120FFF7AAFE040002D0D7
:10C5D0000AE0072070BDFFF79FFE0646FFF7BAFF8F
:10C5E0002A463146FFF7D0FF204670BD405800284C
:10C5F00000D001207047000070B501240B49600491
:10C6000008600B4940108860094940398860094D2D
:10C610006C602F20FFF7CAFDAC60074D00242F206F
:10C62000AC60FFF7C3FDAC7070BD000080E100E0BE
:10C630004013014000100140D4130020F8B5074614
:10C64000012000250C460A26009079192246002078
:10C65000FEF704FF2D18241A002801D1761E01D000
:10C66000002CF2D10098F8BDFEB51F4C0025A7683C
:10C67000606802906846FFF7CBFB0190FFF790FCE3
:10C6800006460198002822D000230098616817E030
:10C690000E680A46864202D9301A086012E0801BF2
:10C6A000F31800261660D668D169B446002E07D06C
:10C6B000FE183602360A566066469660D561154603
:10C6C0000029E5D128466160FFF7C0FC06E0284656
:10C6D000FFF7BCFC002801D1002E02D00298FFF722
:10C6E00043FB0020E070FEBDD4130020012002496E
:10C6F000000508607047000000E200E010B50E4B36
:10C700005968002906D002680C68A24204D8A21A0F
:10C710000A60C161586010BD0B4604E00B46C96950
:10C72000121B002904D00C689442F7D3A41A0C60A1
:10C730000260C161D86110BDD4130020F8B51D4D51
:10C740006C68002C34D01C4800274068A968401A47
:10C750000602360A2068B04218D8361AC71922468F
:10C76000107CE46900280FD000201074EB68002BC7
:10C7700007D0916950699847002805D0FFF718FA4B
:10C7800002E0516990698847002CE3D129786878E4
:10C79000814206D1401CC0B26870022801D100203D
:10C7A000687004490006800D18310F50FFF79EFF96
:10C7B000F8BD0000D41300200015014010B5144648
:10C7C00002460120002A09D00846126805A1FEF79A
:10C7D00061FF01462046FFF7A1FA10BD002121604C
:10C7E00010BD00005B253038645D00000146032069
:10C7F000CA0701D0412040028A0700D502484907F4
:10C8000001D50148401C704701820000FFB50C466D
:10C8100085B000210491FF21053100261F46665096
:10C82000FF2125316650FF211D316650FF2109315E
:10C83000665005462035E11DFF31AE71FA31EE70CC
:10C84000012F0FD001220A600121216221600168BD
:10C85000002909D014498160806803210902611808
:10C8600048601DE00222EEE70146263123300391A5
:10C870000290009701962046079B039A029900F0C8
:10C880002CF80028F5D1E878002809D00920C0014B
:10C890002118486C4864002802D0FFF7A7FF0490D5
:10C8A000049809B0F0BD00008602000030B51C7885
:10C8B000039D944208D205221202095D8018C161CD
:10C8C0001878401C187006E00121002D02D0C161CB
:10C8D000002030BD4161012030BDFFB50F46097811
:10C8E00083B00446002904D1059802780C9882424E
:10C8F00001D1012000E000200190FF20253000251B
:10C90000002907D02550FF201D302550FF20093079
:10C91000255055E0FF2125312046FFF767FE01260F
:10C9200000282CD1FF211D312046FFF75FFE002893
:10C9300014D0FF201D302550FF2125312046FFF760
:10C9400055FE00281BD10D9800902046059B0C9A9F
:10C950000699FFF7ABFF00283FD031E0FF210931F6
:10C960002046FFF743FE00282AD0FF20093025503B
:10C97000FF2125312046FFF739FE002805D0FF2092
:10C980002530255066613E701AE005990C980F78A5
:10C99000069ABC46874213D205231B02E3189B6903
:10C9A0006746D3550A78521CD2B20A70411E8A4299
:10C9B00003D102200102085101E0824200D0266228
:10C9C000019800280BD0FF26053631462046FFF798
:10C9D0000DFE002803D0A551002007B0F0BD0120B6
:10C9E000FBE70000FFB5054687B00C460020FF219D
:10C9F000109F053105906050FF2125316050FF21C7
:10CA00001D316050FF2109316050012149022E463D
:10CA100008512036B071F07001202062A060B31D73
:10CA20000097029320460A9A0999FFF73FFF28686A
:10CA3000002807D01148A860A868032109026118DE
:10CA4000486018E023350A9800900197294620464F
:10CA5000099B029AFFF741FF0028F4D1F0780028E3
:10CA600009D00920C0012118486C4864002802D070
:10CA7000FFF7BCFE059005980BB0F0BD86020000E4
:10CA800010B509494B788C785A1CD2B2944200D127
:10CA900000220C78944201D1002010BD0270486839
:10CAA00018214B43C01810BDE4130020F8130020D8
:10CAB00015161718D4CA0100C81300203000000052
:10CAC000D6B6010004CB0100F8130020B00E000020
:10CAD000E6B60100000000000000000000000000B9
:10CAE0000000000000000000000000000000000046
:10CAF0000000000000000000000000000000000036
:04CB00000024F40019
:040000050001B0C185
:00000001FF
